:100000000CC024C023C022C021C020C01FC01EC0FD
:1000100088C01CC08B9AA4AFB90011241FBECFE9C1
:10002000CDBF10E0A0E6B0E0E2E3F3E002C005904F
:100030000D92AA36B107D9F710E0AAE6B0E001C0E8
:100040001D92AD38B107E1F79CD071C1D9CF28EE30
:1000500033E003C0F9013197F1F70197D8F708951C
:1000600020916B00922F9F5F9F7190936B009EBBBE
:100070008DBB84E28CBB86E28CBBE199FECF2EBBAC
:1000800084E18CBB86E18CBB089540E250E060E0E7
:1000900070E08DE690E03CD180916B0001C08F5FF5
:1000A000E82FF0E0E359FF4F90819F3F19F4803231
:1000B000B0F307C080936B00803218F490936A000D
:1000C000089510926B00089580916A008F5F80936D
:1000D0006A0080916A008A3010F010926A000895D8
:1000E000F894A89581B5886181BD85E481BD789437
:1000F0000895F894A89584B7877F84BF81B58861F7
:1001000081BD11BC7894089581E687B9A29A86ECE6
:1001100086B9089537980895369A3699FECF85B1F5
:1001200008951F920F920FB60F9211242F933F93B1
:100130004F935F936F937F938F939F93AF93BF93EF
:10014000EF93FF9380916C008F3F19F08F5F809346
:100150006C0080916C00823019F480916A0080DF1D
:10016000FF91EF91BF91AF919F918F917F916F918F
:100170005F914F913F912F910F900FBE0F901F9065
:10018000189582E087BB83E28FBD81E083BFBCDF2F
:10019000479A85B7877E85BF78DF80916A0086FFA2
:1001A00006C080916A008F7380936A008DDF809112
:1001B0006A00806455DF94DFE0916A00F0E0E05A65
:1001C000FF4F808189BDA8DFC0E087E2F82E0FEFE6
:1001D00080916A00853040F485B7806285BF88953C
:1001E00085B78F7D85BF58C080916A008830D0F474
:1001F000D4E0E0916A00F0E0E35AFF4F808189BDCE
:1002000085E090E024DFE0916A00F0E0E05AFF4FE3
:10021000808189BD81E490E01ADFD15051F780EDF3
:1002200092E039C080916A00893080F409BD81E094
:1002300090E00DDF19BC89EF90E009DF09BD81E096
:1002400090E005DF19BC8DEE92E025C080916A0038
:100250008A3010F519BC88EE93E0F9DE5DDF5CDFD3
:10026000E4E1F0E0D0E09491981708F4DF5F319674
:1002700090E0E931F907B9F710E009C0F9BC84E66C
:1002800090E0E5DE19BC80E991E0E1DE1F5F1D131F
:10029000F5CF88EE93E0DBDE349B9ACF3DDF90E034
:1002A00020916A00211103C021E730E002C02BE752
:1002B00030E0821793074CF5CF5FC33038F180915F
:1002C0006A00882391F080916A00883009F404C0A4
:1002D00080916A00853019F410926A0013C08091F1
:1002E0006A00815080936A000DC019BC02DF85B797
:1002F000877E806185BF85B7806285BF889585B719
:100300008F7D85BF88EE93E0A2DEC0E0369A60CF95
:10031000A82F862FE82FE199FECF1FBA05C0EEBBAC
:10032000E09AE3950DB20D924150C8F70895F89404
:02033000FFCFFD
:0A033200060E2778FF060E27FF27AE
:00000001FF
